:020000040800F2
:10100000EA320E0248414B52433200000000000019
:101010000000000001010000100008183001640FFA
:10102000001E0000000064000100E803DC05D0079A
:101030006400800C000000000E00000000000000B2
:101040000000646661230000000000000000000052
:101050000000000000000000000000000000000090
:101060000000000000000000000000000000000080
:101070000000000000000000000000000000000070
:101080000000000000000000000000000000000060
:101090000000000000000000000000000000000050
:1010A0000000000000000000000000000000000040
:1010B0000000000000000000000000000000000030
:1010C0000000000000000000000000000000000020
:1010D0000000000000000000000000000000000010
:1010E0000000000000000000000000000000000000
:1010F00000000000000000000000000000000000F0
:1011000000000000000000000000000000000000DF
:1011100000000000000000000000000000000000CF
:1011200000000000000000000000000000000000BF
:1011300000000000000000000000000000000000AF
:0811400000001932000000005C
:10140000002000209560000893600008D94800087B
:1014100000000000000000000000000000000000CC
:1014200000000000000000000000000093600008C1
:101430000000000000000000794800086147000833
:1014400091600008916000089160000891600008B8
:1014500091600008916000089160000891600008A8
:1014600091600008D5170008F953000845410008AD
:101470009160000825450008B11700089160000838
:1014800041450008916000089160000891600008E3
:1014900039410008916000089160000891600008DF
:1014A0009160000891600008916000089153000865
:1014B0005D4100089160000891600008916000089B
:1014C000744B75494FF0FF3210B5DA601A61002293
:1014D000DA601A61714A5A6144F601229A6140F653
:1014E0001202DA614FF0E022C2F8081D5A6822F0B9
:1014F00002025A605A681207FCD41A6822F08072FD
:101500001A601A689401FCD4654A13211160654A77
:101510005A601A6842F080721A601A689001FCD50D
:101520005A6842F002025A604FF090424FF0005168
:10153000116240F2222151622221C2F820144FF49C
:101540008051C2F80C14584911605849C2F800146F
:10155000996941F480319961D36843F01003D360F5
:10156000136823F0100313604021142004F0F6FDEB
:1015700080211B2004F0F2FD40211C2004F0EEFD30
:101580008021092004F0EAFD80210A2004F0E6FD14
:1015900040210B2004F0E2FD0D2004F0C7FD0E20D9
:1015A00004F0C4FD102004F0C1FD142004F0BEFDC1
:1015B0001B2004F0BBFD1C2004F0B8FD092004F042
:1015C000B5FD0A2004F0B2FD0B2004F0AFFD384B4E
:1015D0000222C3F80C2C2022C3F8082C4FF08042C2
:1015E0006021C2F8041478200121C2F81814C2F84E
:1015F0001C04C2F820142F4AC3F808242E4A40F2D3
:101600006711D162092111601168C907FCD4D3F8B0
:10161000082442F00402C3F80824D3F8082452072F
:10162000FBD44FF48072C3F804244FF0FF32C3F8A8
:101630000C242249C3F810240322C3F834240122C5
:101640000A701F4A92F83400012809D102220A7058
:10165000D3F8342442F04002C3F83424194A1070FD
:101660000A78D3F8344402EB82004FF40C728240C3
:101670002243C3F834240A780232D2B20A70013A03
:101680001205C3F82C24104B104A1A61104A5A61F3
:1016900010BD00BF00100240001400080500060045
:1016A0000020024000C03420FFBFEAEBFAEFFFFF4A
:1016B0000020014001008000001000400E020020C8
:1016C0000000002000020020000002404C240140E5
:1016D0000202002006490B68C3F38502104480F320
:1016E000060023F0FC0343EA80030B60704700BF51
:1016F0000010024000F00303013B022B9ABF054A91
:1017000052F8233000234207034A48BF43F4004302
:10171000D3617047986100080000014010B50C4C7F
:101720004FF48033E3600023E360142004F00AFDEB
:10173000E36943F40033E3614FF090431A6A42F4E3
:1017400080721A625A6A42F080525A6210BD00BF1B
:101750000010024008B50A4B4FF48032DA600022D4
:10176000DA60142004F0EEFC4FF09043DA6822F0C7
:101770003002DA601A6842F030021A6008BD00BF19
:1017800000100240074B9A68D2070AD4064A127822
:10179000DA6040F283529A60A3F56043034AC3F8CB
:1017A00008247047000002400E02002001019E0044
:1017B000064B6FF00202C3F8102CD3F80824D205B0
:1017C00044BF034AC3F80824704700BF002001400B
:1017D0000101DE00194A73B50223536000239360B0
:1017E000A2F560421649174CC2F80814247816482E
:1017F0009C420CBF0125022505F10104418830F807
:101800001460028830F81500104CB4FBF6F404FBA9
:1018100000F04FEA203008BF194640F6D865A0F521
:10182000A0606843614362430913001300911213DF
:101830001946643002F0EAFE02B070BD00000240BA
:1018400001008000000200200202002050FB4A003C
:10185000044B1A68002A04DB0028A2BF024A186061
:1018600010607047480100208001002070B50546D7
:101870000E46002456F8240018B1294604F0D6FA82
:1018800008B9204670BD0134F4E713B50A220C46AE
:1018900001A904F0ABFB019B1B781BB92060012060
:1018A00002B010BD0020FBE710B50446006804F04C
:1018B000B3FA206010BD0000F0B585B00A220446DE
:1018C0000D46642791FBF7F601A9304604F07CFA37
:1018D00001462046FFF7E8FF0D492046FFF7E4FFE9
:1018E00007FB16500A2201A904F06EFA04F0CDFAA3
:1018F000084E0546012D05DD01A92046FFF7D4FF5E
:1019000005B0F0BD31462046FFF7CEFF0135F1E7C7
:1019100074640008766400081FB504460A2208466D
:1019200001A904F051FA01462046FFF7BDFF04B0BB
:1019300010BD0000F0B58DB0464F0190054602AED7
:101940000024394601A804F0A8FA18B954B9204671
:101950000DB0F0BD0378002BF3D001340A2C46F80B
:10196000040BEED13C4902980195FFF77FFF09284F
:1019700001F2B283DFE810F00A0015009800AE0310
:101980006807A70BB30BB80BD10BE60B334901A8C3
:10199000FFF78AFF324901A8FFF786FF019C641B0D
:1019A000D5E7012C41F098832E4C2F4901A8FFF771
:1019B0007BFFA078FFF74CFF014601A8FFF7ACFFC3
:1019C0002A4901A8FFF770FFE17801A8FFF7A4FFFB
:1019D000274901A8FFF768FF211D01A8FFF764FF51
:1019E0002449254C01A8FFF75FFF244B01A8196883
:1019F000FFF792FF23683BB1214901A8FFF754FF8D
:101A0000216801A8FFF788FF1E4901A8FFF74CFFD6
:101A10001D4B01A81968FFF74FFF1C4901A8FFF7EC
:101A200043FF1B4B01A81968FFF746FF194901A89E
:101A3000FFF73AFF184B01A81968FFF76DFF174928
:101A400001A8FFF731FF164B196801A8FFF764FFE3
:101A500014499CE778640008EC6600087D6400087F
:101A6000B066000800000020E56400087464000807
:101A7000F2640008F56400080C0700200807002045
:101A8000FE64000806650008280700200F650008AE
:101A9000BC06002018650008B80600202165000873
:101AA000CC0600207B640008012C41F01583AD4C6E
:101AB000AD4901A8FFF7F8FEAC4901A8FFF7F4FE15
:101AC000217D01A8FFF728FFA94901A8FFF7ECFE37
:101AD000A84901A8FFF7E8FEA44901A8FFF7E4FE22
:101AE000617D01A8FFF718FFA14901A8FFF7DCFEFF
:101AF000A14901A8FFF7D8FE9C4901A8FFF7D4FE31
:101B0000A17D01A8FFF708FF994901A8FFF7CCFEC6
:101B10009A4901A8FFF7C8FE944901A8FFF7C4FE3F
:101B2000E17D01A8FFF7F8FE914901A8FFF7BCFE8F
:101B3000934901A8FFF7B8FE8C4901A8FFF7B4FE4E
:101B4000217E01A8FFF7E8FE894901A8FFF7ACFE56
:101B50008C4901A8FFF7A8FE844901A8FFF7A4FE5D
:101B6000617E01A8FFF7D8FE814901A8FFF79CFE1E
:101B7000854901A8FFF798FE7C4901A8FFF794FE6C
:101B8000A17E01A8FFF7C8FE794901A8FFF78CFEE6
:101B90007E4901A8FFF788FE744901A8FFF784FE7B
:101BA000E17E01A8FFF7B8FE714901A8FFF77CFEAE
:101BB000774901A8FFF778FE6C4901A8FFF774FE8A
:101BC000217F01A8FFF7A8FE694901A8FFF76CFE75
:101BD000704901A8FFF768FE644901A8FFF764FE99
:101BE000617F01A8FFF798FE614901A8FFF75CFE3D
:101BF000694901A8FFF758FE5C4901A8FFF754FEA8
:101C0000A17F01A8FFF788FE594901A8FFF74CFE04
:101C1000624901A8FFF748FE544901A8FFF744FEB6
:101C2000E17F01A8FFF778FE514901A8FFF73CFECC
:101C30005B4901A8FFF738FE4C4901A8FFF734FEC5
:101C400094F8201001A8FFF767FE494901A8FFF7A3
:101C50002BFE544901A8FFF727FE444901A8FFF7CE
:101C600023FE94F8211001A8FFF756FE404901A871
:101C7000FFF71AFE4C4901A8FFF716FE3B4901A8E1
:101C8000FFF712FE94F8221001A8FFF745FE38492D
:101C900001A8FFF709FE454901A8FFF705FE3349F2
:101CA00001A8FFF701FE94F8231001A8FFF734FE06
:101CB0002F4901A8FFF7F8FD3D4901A8FFF7F4FD02
:101CC0002A4901A8FFF7F0FD94F8241001A8FFF7B6
:101CD00023FE274901A8FFF7E7FD364901A8FFF7D2
:101CE000E3FD224901A8FFF7DFFD94F8251001A8C4
:101CF000FFF712FE1E4901A8FFF7D6FD2E4901A8E5
:101D0000FFF7D2FD194901A8FFF7CEFD94F8261080
:101D100001A8FFF701FE164901A8FFF7C5FD2749F5
:101D200001A8FFF7C1FD114901A8FFF7BDFD94F817
:101D3000271001A8FFF7F0FD0D4901A8FFF7B4FD3A
:101D40001F4901A8FFF7B0FD084901A8FFF7ACFD46
:101D500094F8281001A8FFF7DFFD054901A8FFF757
:101D6000A3FD2FE0000000202C6500082965000875
:101D70007B64000830650008356500083C65000894
:101D8000446500084B650008566500086165000859
:101D90006A650008736500087C65000885650008B1
:101DA0008F65000899650008A3650008AD65000807
:101DB000B7650008C2650008CC650008D665000854
:101DC000E0650008AC4901A8FFF76EFDAB4901A82A
:101DD000FFF76AFD618D01A8FFF79EFDA84901A8E4
:101DE000FFF762FDA74901A8FFF75EFDA34901A81F
:101DF000FFF75AFDA18D01A8FFF78EFDA04901A8AC
:101E0000FFF752FDA04901A8FFF74EFD9B4901A82D
:101E1000FFF74AFDE18D01A8FFF77EFD984901A873
:101E2000FFF742FD994901A8FFF73EFD934901A83C
:101E3000FFF73AFD218E01A8FFF76EFD904901A83A
:101E4000FFF732FD924901A8FFF72EFD8B4901A84B
:101E5000FFF72AFD618E01A8FFF75EFD884901A802
:101E6000FFF722FD8B4901A8FFF71EFD834901A85A
:101E7000FFF71AFD94F8341001A8FFF74DFD8049D3
:101E800001A8FFF711FD844901A8FFF70DFD7B496B
:101E900001A8FFF709FD94F8351001A8FFF73CFDF4
:101EA000774901A8FFF700FD7C4901A8FFF7FCFC7A
:101EB000724901A8FFF7F8FC94F8361001A8FFF763
:101EC0002BFD6F4901A8FFF7EFFC754901A8FFF74B
:101ED000EBFC6A4901A8FFF7E7FC94F8371001A86A
:101EE000FFF71AFD664901A8FFF7DEFC6D4901A85E
:101EF000FFF7DAFC614901A8FFF7D6FC94F8381027
:101F000001A8FFF709FD5E4901A8FFF7CDFC66496E
:101F100001A8FFF7C9FC594901A8FFF7C5FC618F6B
:101F200001A8FFF7F9FC564901A8FFF7BDFC5F497E
:101F300001A8FFF7B9FC514901A8FFF7B5FC94F8D7
:101F40003C1001A8FFF7E8FC4D4901A8FFF7ACFCE5
:101F5000574901A8FFF7A8FC484901A8FFF7A4FCCE
:101F600094F83D1001A8FFF7D7FC454901A8FFF7F9
:101F70009BFC504901A8FFF797FC404901A8FFF7D7
:101F800093FC94F83E1001A8FFF7C6FC3C4901A859
:101F9000FFF78AFC484901A8FFF786FC374901A8EA
:101FA000FFF782FC94F83F1001A8FFF7B5FC344915
:101FB00001A8FFF779FC414901A8FFF775FC2F49FB
:101FC00001A8FFF771FCB4F8401001A8FFF7A4FCCA
:101FD0002B4901A8FFF768FC394901A8FFF764FC09
:101FE000264901A8FFF760FC04F1420101A8FFF7B0
:101FF0005BFC234901A8FFF757FC324901A8FFF712
:1020000053FC1E4901A8FFF74FFC94F8421101A8A8
:10201000FFF782FC1A4901A8FFF746FC2A4901A8EC
:10202000FFF742FC154901A8FFF73EFC94F8431165
:1020300001A8FFF771FC124901A8FFF735FC2349FD
:1020400001A8FFF731FC0D4901A8FFF72DFC94F81A
:10205000441101A8FFF760FC094901A8FFF724FC1F
:102060001B4901A8FFF720FC044901A8FFF71CFC4D
:1020700094F84511E9E400BFEA6500082965000805
:102080007B640008F4650008FE6500080866000827
:10209000136600081E6600082966000834660008FA
:1020A0003F6600084A660008566600086166000838
:1020B0006B660008756600087F6600088A6600087F
:1020C000946600089A660008A1660008A8660008E1
:1020D000AC660008022C40F0FF8797490398FFF791
:1020E000C5FB292800F2F887DFE810F02A003F003E
:1020F0005200650078008B009E00B100C400D7003C
:10210000EA00FD00100148015D01720187019C0198
:10211000B101C601DB01F0010302160229023C02F3
:102120004F0264027902B402C902DE02F102060320
:102130001B033003450389075A036F038403990384
:102140007E497F4C01A8FFF7AFFB7E4901A8FFF74E
:10215000ABFB217D01A8FFF7DFFB01A87A49FFF760
:10216000A3FB207DFFF774FB14E47849744C01A8AD
:10217000FFF79AFB734901A8FFF796FB617D01A861
:10218000FFF7CAFB01A87049FFF78EFB607DE9E706
:102190006F496B4C01A8FFF787FB6A4901A8FFF75D
:1021A00083FBA17D01A8FFF7B7FB01A86649FFF7F4
:1021B0007BFBA07DD6E76749614C01A8FFF774FB64
:1021C000604901A8FFF770FBE17D01A8FFF7A4FBC0
:1021D00001A85D49FFF768FBE07DC3E75E49584C05
:1021E00001A8FFF761FB574901A8FFF75DFB217EBE
:1021F00001A8FFF791FB01A85349FFF755FB207E8B
:10220000B0E756494E4C01A8FFF74EFB4D4901A8D7
:10221000FFF74AFB617E01A8FFF77EFB01A84A4950
:10222000FFF742FB607E9DE74D49454C01A8FFF753
:102230003BFB444901A8FFF737FBA17E01A8FFF74C
:102240006BFB01A84049FFF72FFBA07E8AE74549B9
:102250003B4C01A8FFF728FB3A4901A8FFF724FBF4
:10226000E17E01A8FFF758FB01A83749FFF71CFBE7
:10227000E07E77E73C49324C01A8FFF715FB314976
:1022800001A8FFF711FB217F01A8FFF745FB01A87B
:102290002D49FFF709FB207F64E73449284C01A84A
:1022A000FFF702FB274901A8FFF7FEFA617F01A8AB
:1022B000FFF732FB01A82449FFF7F6FA607F51E7E8
:1022C0002B491F4C01A8FFF7EFFA1E4901A8FFF7A1
:1022D000EBFAA17F01A8FFF71FFB01A81A49FFF73E
:1022E000E3FAA07F3EE72349154C01A8FFF7DCFA8B
:1022F000144901A8FFF7D8FAE17F01A8FFF70CFB0A
:1023000001A81149FFF7D0FAE07F2BE71A490C4CDE
:1023100001A8FFF7C9FA0B4901A8FFF7C5FA94F81D
:10232000201001A8FFF7F8FA01A80749FFF7BCFA47
:1023300094F8200016E700BF186700082C65000815
:1023400000000020296500087B6400083065000853
:10235000356500083C650008446500084B650008C9
:1023600056650008616500086A6500087365000825
:102370007C650008856500088F650008A249A34CAC
:1023800001A8FFF791FAA24901A8FFF78DFA94F886
:10239000211001A8FFF7C0FA01A89E49FFF784FAAF
:1023A00094F82100DEE69C49984C01A8FFF77CFADE
:1023B000974901A8FFF778FA94F8221001A8FFF7CF
:1023C000ABFA01A89349FFF76FFA94F82200C9E627
:1023D00092498E4C01A8FFF767FA8D4901A8FFF7D3
:1023E00063FA94F8231001A8FFF796FA01A8894927
:1023F000FFF75AFA94F82300B4E68949834C01A800
:10240000FFF752FA824901A8FFF74EFA94F8241018
:1024100001A8FFF781FA01A87E49FFF745FA94F871
:1024200024009FE67F49794C01A8FFF73DFA7849DF
:1024300001A8FFF739FA94F8251001A8FFF76CFA04
:1024400001A87449FFF730FA94F825008AE6764926
:102450006E4C01A8FFF728FA6D4901A8FFF724FA8E
:1024600094F8261001A8FFF757FA01A86949FFF769
:102470001BFA94F8260075E66C49644C01A8FFF736
:1024800013FA634901A8FFF70FFA94F8271001A87F
:10249000FFF742FA01A85F49FFF706FA94F8270010
:1024A00060E66349594C01A8FFF7FEF9584901A8B5
:1024B000FFF7FAF994F8281001A8FFF72DFA01A800
:1024C0005449FFF7F1F994F828004BE659494F4C6D
:1024D00001A8FFF7E9F94E4901A8FFF7E5F9618D79
:1024E00001A8FFF719FA01A84A49FFF7DDF9608D45
:1024F00038E65149454C01A8FFF7D6F9444901A8EF
:10250000FFF7D2F9A18D01A8FFF706FA01A841490A
:10251000FFF7CAF9A08D25E648493C4C01A8FFF712
:10252000C3F93B4901A8FFF7BFF9E18D01A8FFF707
:10253000F3F901A83749FFF7B7F9E08D12E64049F2
:10254000324C01A8FFF7B0F9314901A8FFF7ACF907
:10255000218E01A8FFF7E0F901A82E49FFF7A4F9A1
:10256000208EFFE53749294C01A8FFF79DF928493E
:1025700001A8FFF799F9618E01A8FFF7CDF901A82D
:102580002449FFF791F9608EECE52F491F4C01A813
:10259000FFF78AF91E4901A8FFF786F994F834106D
:1025A00001A8FFF7B9F901A81A49FFF77DF994F8D6
:1025B0003400D7E52549154C01A8FFF775F91449F2
:1025C00001A8FFF771F994F8351001A8FFF7A4F9F5
:1025D00001A81049FFF768F994F83500C2E51C49D5
:1025E0000A4C01A8FFF760F9094901A8FFF75CF957
:1025F00094F8361001A8FFF78FF901A80549FFF7F5
:1026000053F994F83600ADE5996500080000002004
:10261000296500087B640008A3650008AD65000813
:10262000B7650008C2650008CC650008D6650008DB
:10263000E0650008EA650008F4650008FE6500082A
:1026400008660008136600081E6600082966000870
:1026500034660008A249A34C01A8FFF725F9A24956
:1026600001A8FFF721F994F8371001A8FFF754F9F2
:1026700001A89E49FFF718F994F8370072E59C49C4
:10268000984C01A8FFF710F9974901A8FFF70CF93A
:1026900094F8381001A8FFF73FF901A89349FFF714
:1026A00003F994F838005DE592498E4C01A8FFF7D4
:1026B000FBF88D4901A8FFF7F7F8618F01A8FFF734
:1026C0002BF901A88949FFF7EFF8608F4AE58A499D
:1026D000844C01A8FFF7E8F8834901A8FFF7E4F864
:1026E00094F83C1001A8FFF717F901A87F49FFF7FC
:1026F000DBF894F83C0035E580497A4C01A8FFF7F7
:10270000D3F8794901A8FFF7CFF894F83D1001A854
:10271000FFF702F901A87549FFF7C6F894F83D00E4
:1027200020E577496F4C01A8FFF7BEF86E4901A874
:10273000FFF7BAF894F83E1001A8FFF7EDF801A8EA
:102740006A49FFF7B1F894F83E000BE56D49654C16
:1027500001A8FFF7A9F8644901A8FFF7A5F894F8C4
:102760003F1001A8FFF7D8F801A86049FFF79CF8CF
:1027700094F83F00F6E464495A4C01A8FFF794F836
:10278000594901A8FFF790F8B4F8401001A8FFF7E5
:10279000C3F801A85549FFF787F8B4F84000E1E411
:1027A0005A49504C01A8FFF77FF84F4901A8FFF79D
:1027B0007BF894F8421101A8FFF7AEF801A84B4945
:1027C000FFF772F894F84201CCE45149454C01A856
:1027D000FFF76AF8444901A8FFF766F894F8431137
:1027E00001A8FFF799F801A84049FFF75DF894F8B0
:1027F0004301B7E447493B4C01A8FFF755F83A4974
:1028000001A8FFF751F894F8441101A8FFF784F8E4
:1028100001A83649FFF748F894F84401A2E43E497C
:10282000304C01A8FFF740F82F4901A8FFF73CF80A
:1028300094F8451101A8FFF76FF801A82B49FFF79D
:1028400033F894F845018DE4032C40F04584334976
:102850000398FFF70BF8292800F23E84DFE810F018
:102860002A00620077008C00A100B600CB00E000D7
:10287000F5000A011F0134014901600176018C0154
:10288000A201B801F4010B02220239024F026502D3
:102890007B029102A702BE02D502EC0202031903D9
:1028A0002F03460382039903B003C703DD03F30339
:1028B00009041E0404986946FEF7E7FF002800F0AB
:1028C0000B84084C009B237502F020FF01A81449DB
:1028D000FEF7EAFF044901A8FEF7E6FF39E400BF6E
:1028E0003F66000800000020296500087B6400089E
:1028F0004A66000856660008616600086B660008B4
:10290000756600087F6600088A6600089A660008F7
:10291000A1660008A8660008AC66000818670008F1
:102920002C65000804986946FEF7AFFF002800F008
:10293000D383B24C009B637502F0E8FE01A8B04956
:10294000FEF7B2FFAF4901A8FEF7AEFF16E4049808
:102950006946FEF79AFF002800F0BE83A74C009B53
:10296000A37502F0D3FE01A8A749FEF79DFFA54974
:1029700001A8FEF799FF14E404986946FEF785FF65
:10298000002800F0A9839D4C009BE37502F0BEFE79
:1029900001A89E49FEF788FF9A4901A8FEF784FF27
:1029A00012E404986946FEF770FF002800F0948353
:1029B000924C009B237602F0A9FE01A89449FEF7F1
:1029C00073FF904901A8FEF76FFF10E40498694671
:1029D000FEF75BFF002800F07F83884C009B637646
:1029E00002F094FE01A88B49FEF75EFF854901A81D
:1029F000FEF75AFF0EE404986946FEF746FF0028EA
:102A000000F06A837D4C009BA37602F07FFE01A854
:102A10008149FEF749FF7B4901A8FEF745FF0CE419
:102A200004986946FEF731FF002800F05583734C87
:102A3000009BE37602F06AFE01A87849FEF734FFB6
:102A4000704901A8FEF730FF0AE404986946FEF7D2
:102A50001CFF002800F04083684C009B237702F0A5
:102A600055FE01A86E49FEF71FFF664901A8FEF753
:102A70001BFF08E404986946FEF707FF002800F0F2
:102A80002B835E4C009B637702F040FE01A86549F2
:102A9000FEF70AFF5B4901A8FEF706FF06E404986B
:102AA0006946FEF7F2FE002800F01683534C009BA7
:102AB000A37702F02BFE01A85B49FEF7F5FE514912
:102AC00001A8FEF7F1FE04E404986946FEF7DDFE76
:102AD000002800F00183494C009BE37702F016FECA
:102AE00001A85249FEF7E0FE464901A8FEF7DCFEC8
:102AF00002E404986946FEF7C8FE002800F0EC8264
:102B00003E4C009B84F8203002F000FE01A84849AA
:102B1000FEF7CAFE3B4901A8FEF7C6FEFFF7FFBB62
:102B200004986946FEF7B1FE002800F0D582334CC8
:102B3000009B84F8213002F0E9FD01A83D49FEF731
:102B4000B3FE304901A8FEF7AFFE20E404986946C1
:102B5000FEF79BFE002800F0BF82284C009B84F803
:102B6000223002F0D3FD01A83349FEF79DFE25492E
:102B700001A8FEF799FE1FE404986946FEF785FE5A
:102B8000002800F0A9821D4C009B84F8233002F03D
:102B9000BDFD01A82949FEF787FE1A4901A8FEF7E5
:102BA00083FE1EE404986946FEF76FFE002800F0DD
:102BB0009382124C009B84F8243002F0A7FD01A8F8
:102BC0001F49FEF771FE0F4901A8FEF76DFE1DE4D7
:102BD00004986946FEF759FE002800F07D82074CF4
:102BE000009B84F8253002F091FD01A81549FEF7FD
:102BF0005BFE044901A8FEF757FE1CE4000000201C
:102C00003065000829650008356500083C65000846
:102C1000446500084B6500085665000861650008BA
:102C20006A650008736500087C6500088565000812
:102C30008F65000899650008A3650008AD65000868
:102C4000B7650008C265000804986946FEF71DFED6
:102C5000002800F04182B14C009B84F8263002F03D
:102C600055FD01A8AE49FEF71FFEAE4901A8FEF7CB
:102C70001BFEFFF7F5BB04986946FEF706FE002829
:102C800000F02A82A54C009B84F8273002F03EFD1C
:102C900001A8A549FEF708FEA24901A8FEF704FE17
:102CA000FFF7F3BB04986946FEF7EFFD002800F03C
:102CB00013829A4C009B84F8283002F027FD01A86B
:102CC0009A49FEF7F1FD974901A8FEF7EDFDFFF7E0
:102CD000F1BB04986946FEF7D8FD002800F0FC819E
:102CE0008E4C009B638502F011FD01A89049FEF710
:102CF000DBFD8C4901A8FEF7D7FDFFF7F0BB049878
:102D00006946FEF7C2FD002800F0E681834C009B77
:102D1000A38502F0FBFC01A88649FEF7C5FD8149A9
:102D200001A8FEF7C1FDFFF7EDBB04986946FEF769
:102D3000ACFD002800F0D081784C009BE38502F0C8
:102D4000E5FC01A87C49FEF7AFFD764901A8FEF736
:102D5000ABFDFFF7EABB04986946FEF796FD002835
:102D600000F0BA816D4C009B238602F0CFFC01A8D5
:102D70007249FEF799FD6B4901A8FEF795FDFFF733
:102D8000E7BB04986946FEF780FD002800F0A481A7
:102D9000624C009B638602F0B9FC01A86849FEF70B
:102DA00083FD604901A8FEF77FFDFFF7E4BB0498AF
:102DB0006946FEF76AFD002800F08E81574C009BA3
:102DC00084F8343002F0A2FC01A85E49FEF76CFDE5
:102DD000544901A8FEF768FDFFF7E0BB0498694677
:102DE000FEF753FD002800F077814C4C009B84F8DF
:102DF000353002F08BFC01A85349FEF755FD4949D7
:102E000001A8FEF751FDFFF7DEBB04986946FEF707
:102E10003CFD002800F06081404C009B84F8363077
:102E200002F074FC01A84949FEF73EFD3D4901A8A6
:102E3000FEF73AFDFFF7DCBB04986946FEF725FD77
:102E4000002800F04981354C009B84F8373002F0AF
:102E50005DFC01A83E49FEF727FD324901A8FEF7B7
:102E600023FD00E404986946FEF70FFD002800F0FA
:102E700033812A4C009B84F8383002F047FC01A8CB
:102E80003449FEF711FD274901A8FEF70DFDFFF7B4
:102E9000FFBB04986946FEF7F8FC002800F01C818F
:102EA0001E4C009B638702F031FC01A82A49FEF703
:102EB000FBFC1C4901A8FEF7F7FCFFF7FEBB0498DA
:102EC0006946FEF7E2FC002800F00681134C009BE7
:102ED00084F83C3002F01AFC01A82049FEF7E4FC1B
:102EE000104901A8FEF7E0FCFFF7FABB0498694619
:102EF000FEF7CBFC002800F0EF80084C009B84F824
:102F00003D3002F003FC01A81549FEF7CDFC054950
:102F100001A8FEF7C9FCFFF7F8BB00BF00000020C6
:102F2000CC65000829650008D6650008E065000842
:102F3000EA650008F4650008FE65000808660008F8
:102F4000136600081E66000829660008346600083B
:102F50003F6600084A660008566600086166000879
:102F60006B66000804986946FEF78FFC002800F0A5
:102F7000B3807B4C009B84F83E3002F0C7FB01A875
:102F80007849FEF791FC784901A8FEF78DFCFFF720
:102F9000D1BB04986946FEF778FC002800F09C80BD
:102FA0006F4C009B84F83F3002F0B0FB01A86F49E2
:102FB000FEF77AFC6C4901A8FEF776FCFFF7CFBB61
:102FC00004986946FEF761FC002800F08580644C97
:102FD000009BA4F8403002F099FB01A86449FEF779
:102FE00063FC614901A8FEF75FFCFFF7CDBB0499C4
:102FF00060484FF4807202F033FF02F087FB01A8B3
:103000005D49FEF751FC01A85749FEF74DFC5949AF
:1030100001A8FEF749FCFEF71BBD04986946FEF7C0
:1030200034FC002858D04E4C009B84F8423102F00A
:103030006DFB01A85149FEF737FC4B4901A8FEF78B
:1030400033FCFFF7B6BB04986946FEF71EFC002868
:1030500042D0434C009B84F8433102F057FB01A857
:103060004749FEF721FC404901A8FEF71DFCFFF788
:10307000B5BB04986946FEF708FC68B3384C009B62
:1030800084F8443102F042FB01A83E49FEF70CFCF3
:10309000354901A8FEF708FCFFF7B5BB049869465F
:1030A000FEF7F3FBC0B12E4C009B84F8453102F0D3
:1030B0002DFB01A83449FEF7F7FB2B4901A8FEF7C9
:1030C000F3FBFFF7B5BB012C06D102F0ABFCFEF71A
:1030D000BFFB00287EF45EAC2C49FEF75CBC012CE3
:1030E000FAD102F0EBFCF2E7A31E012BF4D81C4B43
:1030F000032C93F84231009304D00099039802F016
:1031000001FDE6E704986946FEF7BFFB0028E3D01F
:10311000009B013B632BF0D9DEE7022CDCD1039846
:103120006946FEF7B2FB0028D6D0009B03F5FA6291
:10313000B2F57A6FD0D8164A1360164B00221A7077
:10314000FEF728BC012CC7D1134B1A68002ABCBF5C
:1031500000221A601A68114B1A60FEF71BBC00BFF0
:103160000000002075660008296500087F660008D9
:103170008A66000842000020946600089A660008EB
:10318000A1660008A8660008AC660008B4660008DE
:103190001007002098060020480100208001002030
:1031A000114B00214FF48032DA60D960A3F550430F
:1031B0004FF400425A6481221A600C4A91650C490E
:1031C00051662021D16540F2A35191654FF0FF3245
:1031D000DA62442101225A619960332199611A62AD
:1031E0004FF40072DA6070470010024000000240A5
:1031F0002402002008B50B4B1B780BB1FFF7D0FF62
:10320000094B00229A65A3F5404385221A60074ABC
:103210001288DA626FF0010101225A611961DA60E5
:1032200008BD00BF64020020000002402002002010
:103230004FF04023D3F80024D3F80424D3F80C240F
:1032400042F01002C3F80C240822C3F8142403F53A
:10325000E03300229A6570470A4B6FF001021A6151
:103260000022DA604FF0FF32DA6201225A614FF039
:10327000402343F20C42C3F80C24034B034A1A6068
:10328000704700BF0040014070060020F138000880
:1032900029482A4B01686FF00102F0B5284D1A61E8
:1032A000052945D8DFE801F00327292F3335254BC1
:1032B0001B6864331A1242F0800295F83750224C92
:1032C0006E1E224D6370062707FB0655204B6D5C72
:1032D000A27025700131002203245A6405299C64E0
:1032E0004FF091045C64C8BF1A4B0160C2BF1A4919
:1032F00019600260F0BD194BDAE7194B1A68131216
:1033000043F04003D9E7174B1A681312D5E7164B61
:10331000FAE795F83830154A03EB4303126892FB3D
:10332000F3F34FF6FF729342A8BF13461A12C4E795
:1033300000221346C1E700BF800600200040014084
:1033400000000020080700206C020020D46700085D
:103350000000024070060020593200080C070020CF
:10336000BC06002028070020B8060020CC0600205C
:1033700037B5144C94F82430C3B1A18DA1F13202B9
:1033800082420ADD0023618D0093A3F5FA6302F007
:103390007DF90D4B186003B030BD323181420DDA3A
:1033A0004FF4FA6300930023E28DF0E7618D323130
:1033B000814205DA4FF4FA620092F5E70020E8E76F
:1033C0001846E6E70000002010070020F0B4184B74
:1033D00093F835200B23013A02EB42045A43D210F2
:1033E00004F007050334865C04F007048118012308
:1033F000A340A5424A7846FA05F6C5F1080703F14D
:10340000FF300BDA024002FA07F0304300EB800095
:10341000C010F0BC00F55C70FFF7AABF8B78C5F157
:103420001005034002FA07F0AB4030431843EDE7C4
:10343000000000204FF04022C820D2F80034D2F81B
:103440000434134B10B5D96DC2F8140442F21C00B9
:10345000C2F80C0400229A654022DA6526294FF052
:1034600081029A6513D10B4C617818290FD1A3788A
:10347000162B0CD1A01C02F0F9F840B9064B4AF605
:10348000AA22E01C1A60BDE81040FFF79FBF10BDE4
:10349000000002406C020020003000400E4B5A6BCE
:1034A000986BB2F5FA6F16DBA0F11C03042B07D85A
:1034B0000A4B4AF6AA221A60094B01221A70704779
:1034C000A0F54873B3F5AF6F05D8044B4AF6AA22AE
:1034D0001A60FFF74DBF70470040014000300040C8
:1034E0000507002010B5054C207000126070022105
:1034F000204602F0ABF8A070032010BD6C02002043
:1035000010B43E4A3E4B92F828205B6B002A65D0EF
:10351000A3F5A542013A40F2DE618A4231D9A3F512
:103520009642013A40F23E618A422AD9A3F52552D9
:10353000013A40F26E318A4223D9A3F51652013A7C
:1035400040F21E318A421CD9A3F5F052013A40F2F2
:103550007E218A4215D9A3F59652013AB2F5C77F6A
:103560000FD96FF470601A18B2F59F7F09D96FF404
:1035700034615A18EE2A04D96FF4F0629A189E2A20
:103580002CD8204A20484AF6AA2111601F4903F589
:10359000FA7292FBF1F24FF47A7101FB02331C498B
:1035A0000A68134402680B600132026012F00302E1
:1035B00022D118480468A342174C07DD5B42236000
:1035C0000A604FF0FF3010BCFEF784B82468A342B5
:1035D00004DA5B4203600A600120F4E70F4B104AF3
:1035E0001A60074B49F291229A6131221A626FF0F8
:1035F00004021A610422DA6010BC70470000002047
:1036000000400140003000407C06002018FCFFFF15
:1036100084060020900600209406002070060020FA
:103620009D340008F8B57F4B1A6912F001022FD0C3
:103630006FF001021A614FF090431B6913F004030D
:103640000DD1794A92F83420012A05D1FEF782F88B
:10365000764B01221A70F8BD754A1360FBE7754A74
:10366000136801330F2B1360F5DD734B734A1A6037
:10367000FEF754F84FF040230822C3F8142440F614
:103680003542C3F8082442F22C02C3F80C24E2E7C6
:10369000654E596B96F83440012CD7D064480768C2
:1036A0007D1C0560002FD6D0654F4CF6CC4C012C0C
:1036B000C7F800C060D9604C624B2360FEF72EF85B
:1036C00096F83430023B032B3AD8DFE803F0020FC0
:1036D0001A4E5D4B5D4A1A605D4B04221A704FF022
:1036E00040234FF48272C3F8082429E0564B594A0C
:1036F0001A60574B20221A704FF0402340F21242BA
:10370000F1E7514B544A1A60514B19221A704FF08D
:1037100040234FF49662C3F808244FF4A052C3F834
:103720000C244FF40052C3F8102403F580330E220A
:103730009A624FF0FF32DA6201225A6181221A60E6
:103740004FF040220823C2F81434D2F80C34434915
:1037500043F4005343F01C03C2F80C34404B414A7D
:1037600019665A66D9641A6575E73F4B23604FF4B2
:1037700090724FF04023B6E79E6A0C46F6B1B1F561
:10378000FA6F06DD2C4B394A1A60BDE8F840FFF7A6
:10379000B7BE996A772908BF0E229A6201225A6140
:1037A0000023036057E764100139952CFBDC304B94
:1037B0001A688A4204D019600123F2E70221F4E773
:1037C0000029FFF648AF032D7FF745AF1A4B294A72
:1037D0001A601D4B284A29481A60294A884002EB82
:1037E0006003B3FBF0F32748013B9BB203802648FC
:1037F00000FA01F102EB6102B2FBF1F22349013A56
:103800000A80084A002111624421916033219161AC
:103810000121D160D362124B516134321A661C4AC5
:103820005A6618E70040014000000020980600207A
:10383000780600201002002070060020ED3A0008F3
:1038400000300040F13800086C0600209D39000867
:103850008C06002039390008B53B000804440040BC
:10386000000002406C0200203534000801350008D9
:103870001C020020953800086D3C0008F049020049
:10388000000E270720020020D8B8050022020020E1
:1038900024020020134BDA68D10722D51A69D20717
:1038A0001FD56FF001021A611A6A42B901221A6229
:1038B0004FF090430C4A1B6903F0040313700B4B49
:1038C0002022DA6540F2A3529A65A3F540434FF0F7
:1038D000FF32DA6201225A6181221A604FF40072CB
:1038E000DA6070470040014064020020000002409E
:1038F0004FF04023D3F80C24520604D542F20C02B8
:10390000C3F80C247047D3F80024D3F80424D3F868
:103910000C2422F01002C3F80C24C822C3F814248B
:10392000034B1A78034BDA65A3229A65704700BFF0
:103930008C06002000000240F0B4154B1A78202AB3
:1039400002D15A78402A02D0F0BCFFF771BC114A6C
:103950004FF69F7492F8357040F2DC50012299784E
:10396000DE780F2A41EA062508D1A542ECD10A4BA0
:103970004AF6AA22F0BC1A60FFF7FABC974231441B
:10398000A4EB010408BFC5F30B0001320233E6E7E4
:103990006C020020000000200030004010B5484CB0
:1039A0000421204601F052FE18B1BDE81040FFF797
:1039B0003FBC444B4AF6AA221A602278B4F8013080
:1039C00002F00F010139184603290ED8DFE801F093
:1039D00002171D24190448BFA3F5803000F5FA63CF
:1039E000B3F57A6F01D8384B18601309083B062BE2
:1039F0005AD8DFE803F0174E5A5D5F616300003B61
:103A0000324918BF01230B70EFE73149642BA8BF7F
:103A1000642381F82230E8E72D4903F0070381F899
:103A20004531E2E72B4B26481B6823702A4B1B6865
:103A300063702A4B1B68A3701B12E370284B1B6832
:103A400023711B126371274B1B68A3711B12E37157
:103A5000254B1B684FF6FF729342A8BF1346237293
:103A60000A211B12637201F0F1FDA0720B204FF0CE
:103A700040236FF04002C3F8002442F24802C3F82A
:103A80000C2403F5E03300225A64912298645A64AE
:103A90000AE0154B18684FF6FF739842A8BF184606
:103AA000FFF720FD0028E2D110BD0A4B1868F7E7A8
:103AB000094BFBE7094BF9E7094BF7E7094BF5E73A
:103AC0006C0200200030004010070020D5060020C6
:103AD00000000020080700200C0700202807002015
:103AE000BC060020B8060020D00600204FF040237E
:103AF00010B5D3F80C24110613D52A4A2A4C1168A4
:103B0000481C615C1060C3F8041428490C68A0428A
:103B100006DB42F24800C3F80C04002313600B607C
:103B200010BD520604D542F22C02C3F80C24F7E76C
:103B3000D3F800241B4912F0060F0B6803D140F2A2
:103B4000FF32934203D11A4A8020C2F8000C4FF092
:103B50004022D2F80424D2B2082A01D07F2A03D10D
:103B6000002BDDD0013BDAE75C1C0F480C60022C17
:103B7000C25406D1037823B94378FF2B01D102F058
:103B8000CDFA0A2ACCD10023035507480B60FDF774
:103B9000D1FE064B18600028C2D04FF0402342F2FD
:103BA0008802C2E7680200206C0200207406002030
:103BB0000020004070B5254D2B780F2B03D0BDE8B9
:103BC0007040FFF735BB224B224C01264AF6AA2251
:103BD0006661A8191A60FFF7F9FB297E01F00F034F
:103BE000042B24D11C4B1D4A1B78023BB34206D93F
:103BF0001B4B93F83730013BB3EB111F18D0194B17
:103C0000136072B6134A536AC3F563437F33D362BA
:103C10000123536162B60F4B6FF001021A6101225A
:103C2000DA604FF0402343F20842C3F80C2470BD21
:103C30000D4B136072B6636AC3F5F8435F33E362FA
:103C40006661636941F29F43E362E3E76C0200202F
:103C500000300040004001400407002070060020B2
:103C6000000000205932000891320008AE498A6DE8
:103C700012F01002F8B548D0AC48FFF791FA02688C
:103C80006AB9AB4B19684FF6807311B18B42A8BF6C
:103C90000B46B3F5007F2EDA43EA42230360036844
:103CA00019011A461B1129D1D24302F00F02A14E6D
:103CB0000A4319468C0042FA04F505F00F050C443E
:103CC000755D013105FA04F4042943EA0403F1D1D6
:103CD000994C13224FF0FF3143FA02F5ED0748BF2C
:103CE000C943013A24F8021FF6D2944A13683BB93B
:103CF00000230360F8BD5B100132CAE75A40D1E7E8
:103D0000013B1360002BF3D0F4E78D4C23780BB309
:103D10008C4B78201A629A609A61986108205860EA
:103D200085488A6548661720C86540F293508865C3
:103D30005A6372B65A6AC2F560620F32132AB8BF6C
:103D40001322DA6201225A6159697F490988D962CE
:103D50001A6262B67D4B7E481988002201318D10AF
:103D6000134647885B00AF4202F10202A8BF43F04E
:103D70000103202A064618D1207819461A4609114F
:103D80001CD100B1D24312F00F0213D171494AF68F
:103D9000AA20086003F010015B1100F084812F2B32
:103DA00011DD002900F084817EE1B6888E4200F1A9
:103DB0000400D6DBBDE8F840FFF71CBA4A40DEE756
:103DC000A3F12F0282E1002994D0594A10680028FB
:103DD00090D161490A689A42604A1CBF0B6010602A
:103DE0001368092BDCBF013313600B68591E2E29A1
:103DF00080D801A050F821F0B53E0008B53E00087B
:103E0000B53E0008B53E0008B53E0008F53C000888
:103E1000BB3E0008CB3E0008D93E0008EB3E000840
:103E2000F53C0008F93E00080B3F0008713F000810
:103E3000F53C0008F53C0008F53C0008F53C00089E
:103E4000F53C0008873F0008973F0008A53F0008A1
:103E5000C13F0008D93F0008F53C0008B53F000805
:103E6000CD3F0008E53F0008F53C0008F53C0008A0
:103E7000F53C0008F53C0008F53C0008F53C00085E
:103E8000F53C0008F53C0008F53C0008F53C00084E
:103E9000F53C0008F13F00081B40000845400008C1
:103EA0006F400008F53C0008F53C0008F53C0008B0
:103EB000994000082A4A13701CE71368062B7FF408
:103EC00019AF284B00229A7514E71368062B7FF46C
:103ED00011AF244B0122F6E71368062B7FF40AAFDB
:103EE000204B002283F8242004E71368062B7FF47C
:103EF00001AF1C4B0122F5E71368062B7FF4FAAEE5
:103F000001F090FD184B1860F4E61368062B7FF45F
:103F1000F1AE164B01221A70044B4FF460621A6026
:103F2000064B0A22D6E000BF00000240C80600206F
:103F3000D0060020C46700084C010020880600203D
:103F400064020020004001402202002020020020E4
:103F5000240200200030004014020020180200203B
:103F6000990600200000002080010020C4060020E7
:103F70001368062B7FF4BEAE574B00221A70574BC6
:103F800040F6FF62CBE71368062B7FF4B3AE544BC9
:103F900000221A70AEE61368062B7FF4ABAE504BCE
:103FA0000122F6E74F4A92F8453143F0010382F8C7
:103FB00045319FE64B4A92F8453123F00103F6E77D
:103FC000484A92F8453143F00203F0E7454A92F837
:103FD000453123F00203EAE7424A92F8453143F0C3
:103FE0000403E4E73F4A92F8453123F00403DEE797
:103FF0001368062B7FF47EAE3A4A137E5B080133CA
:104000000F2B08D8082BB8BF082359001176073B9F
:10401000354A13606EE60823F7E71368062B7FF432
:1040200069AE3049CA7E920801320C2A03D8062AAA
:104030001346B8BF0623DAB29000D200C8760A77DA
:10404000053BE5E71368062B7FF454AE25490A22A9
:1040500091F82030B3FBF2F30133DBB20B2B28BF16
:10406000002303EB8302520081F82020D0E713687D
:10407000062B7FF43FAE1B490A2291F82130B3FB97
:10408000F2F30133DBB20B2B28BF012303EB8302D6
:10409000520081F82120BBE71368062B7FF42AAE7B
:1040A00001F00CFD2EE789B11049012008706BB1B9
:1040B0000C4A92F82420002A3FF482AEB3F5836FB5
:1040C000ACBFA3F21743C3F12F035A00084B1A6089
:1040D000084B00221A600DE6C4060020C806002026
:1040E000D5060020000000208001002005070020E8
:1040F00010070020140200200C4B0D4A1A600D4BD3
:104100004FF400425A6454229A6031229A6103218A
:1041100001221A62D960772199624FF0FF31D9628A
:10412000042119605A6185221A60704770060020C8
:104130002536000800400140014B1B68184700BFAE
:1041400070060020034B4FF400325A60024B1B688C
:10415000184700BF000002406C060020FFF7ECBFCC
:10416000014B01225A61704700100040BC4BBD4911
:104170002DE9F0471E68BC4DBC4C2B68002E75D055
:104180004FF080420120C2F83C64C2F82C64B84E63
:10419000C2F81404327822B91BB13C2253433B3B92
:1041A0002B600A782B68002A54D0013B002BD8BF23
:1041B0004FF4B4732B6029684A1E772A50DC01F152
:1041C000EF077731AB48AC4B05689B7EC5F17805AE
:1041D000DB00AB42A8BF2B4618468323C4F8003C43
:1041E00041F28733C4F82C3CA44B33F812204243ED
:1041F000D2114232C4F8342C33F8172033F811307E
:1042000042434343D211DB1142334232C4F8382CCB
:10421000C4F83C3C8123C4F8003C3578C5B946F667
:104220006803C4F8183C6823C4F81C3C40F255539A
:10423000C4F8203C2123C4F8143C4FF080432846A6
:10424000C3F80C54FDF756FA8D4B1D6001233370F3
:10425000BDE8F0870133B3F5B47FC8BF0123A9E7F8
:10426000EF2AA1F17907ACDDF139ABE70F78002F28
:1042700000F08480013B002BD8BF06232B602B6805
:10428000804A1A4403F0010312F8012C02EAD2001A
:10429000D143BB4218BF042610F0010301EAD2014A
:1042A00071D0754A527D002A18BF052343F480530C
:1042B00040F66802870774D56F4F7F7D002F14BFCB
:1042C0005027102742F4C0423B43400774D56A4947
:1042D000497D002914BF4FF4A0614FF480710B4356
:1042E00046F66801684FC4F8182C3868C4F81C1CDE
:1042F000C4F8203CFDF7FEF93E60644FDFF8809182
:104300003868DFF88C81634EB0F57A7F5FDD624BF1
:104310004FF47A721A600023C8F800303368632BB8
:104320004FF0000273DCC4F8402C4FF08043712240
:10433000C3F818248522C3F800244FF080430022DC
:10434000C3F810240322C3F80C242B68534A39689D
:10435000013B42F82310D9F80030052B7FF778AFE6
:10436000D2E900310B4491680B44D1680B441169C8
:1043700052690B4413445B10336069E70133062B29
:10438000C8BF01237AE7CB075DBF46F0010641F2C3
:10439000040340F6480241F2040348BF40F65802C5
:1043A00088E78F0743F040034EBF42F4A04242F437
:1043B000804246F0020688E7490743F480635ABF0B
:1043C00046F0030646F6480146F658018AE7D8F853
:1043D00000300133062BC8F800309FD1DFF8B8A0B9
:1043E000DAF80030181A01F0CFFC3B68B0EB630F2D
:1043F00009DD2B4A0023C9F80030137041F28833DD
:104400003B60284B33603B68CAF8003083E7C72B1A
:1044100005DCC4F8402C4FF08043912288E7B3F5C7
:104420007A7F05DAC4F8402C4FF08043C1227FE741
:10443000B3F5FA6F4FF0804307DAC4F8402CC1227D
:10444000C3F8182440F2851275E74FF40072C4F8DF
:10445000402CC122C3F8182440F285226BE700BF2C
:10446000F8060020F5060020FC0600200020014090
:10447000EC060020C006002000000020A461000817
:1044800000070020BE690008E8060020DC060020C6
:10449000B4060020D0060020240700209C0600203F
:1044A000D406002000E1F50538B501F019FB1749E5
:1044B000174A0B68174C5BB113784BB123683C204B
:1044C0001D3393FBF0F30133062BC8BF0123236098
:1044D00000230B601370104B104D1B786BB1FFF76E
:1044E00045FE2123C5F8143C0020FDF703F90C4BD1
:1044F00022681A600023236038BD46F66803C5F8B9
:10450000183C6823C5F81C3CEBE700BFF806002008
:10451000EC060020FC060020E00600200020014000
:10452000E4060020054BD3F80C2C920605D56FF05D
:104530002002C3F8102CFFF719BE7047002001407D
:104540004FF0804310B5D3F80C24D3F81014D007E3
:1045500014D5C90712D56FF00102C3F81024002248
:10456000C3F80C24234B1A60234B1A70234B42F2DE
:1045700010721A60224B234A1A6010BD9307FCD5B3
:104580001E484FF080430268D3F83434B3EB620F17
:10459000F3DB02EB4202B3EBA20F02DBB3EB620FE1
:1045A00025DD17490968B1F5FA6FACBF002101217B
:1045B0001344154A104C127E21709B105A4303601D
:1045C000A3EB62135B104FF08042012BB8BF0123B5
:1045D000C2F83C340123C2F814340023C2F80C346E
:1045E000044A1368052BDCBF01331360C5E70021C3
:1045F000DEE700BF00070020D4060020DC06002014
:10460000D006002000E1F5050000002073B501464A
:104610003F48404C164602689B1A67D4012323701A
:104620000A223D4801F044F83C4A831023EAE37330
:10463000136000210A220546394801F039F839494A
:10464000394A831023EAE373714313604914072244
:104650000446364801F02CF8354B0422186000213E
:10466000344801F025F8344B344918600B6818447D
:10467000334B08601A68C2F3090252B9314E0A601E
:10468000336803EBA0235B20336043432E48DB13E6
:1046900003602E4E96F83C3083B196F83D20012AF7
:1046A0004FEA83032BD0022A2BD032B35B4223EA9A
:1046B000E373274A3C2BA8BF3C231360254B1B7890
:1046C00093B106992448052200F0F2FF96F82730AE
:1046D0004FF4FA62009203EB83039B00728E318EDB
:1046E00000F0D4FF1D4B186002B070BD2478002C80
:1046F00096D102EB6302026092E7EB1AD7E7E31A66
:10470000D5E7A542ACBFC3EB0503C3EB0403CEE77B
:1047100098010020F40600208C01002008070020EA
:1047200090010020E43202000C07002094010020D8
:104730002807002088010020BC060020D8060020A1
:1047400018070020F0060020B80600200000002016
:10475000C0060020980600208401002010070020D9
:104760004FF0E0234FF08052C3F8042D0022C3F82D
:10477000102D094A13780133DBB2137013F00F03C5
:1047800009D106490A6801320A60054909688A4266
:1047900004BF044A13707047140700201807002054
:1047A000200700201C07002038B50C4672B6074BC6
:1047B000074D1B681844074B186001232B7062B625
:1047C0002B7803B938BDA047FAE700BF18070020CF
:1047D0001C070020200700202DE9F047204C2378FB
:1047E0008AB053B11F4A013B92F843111E4A52F856
:1047F000230001F087F9002323701C4F3B68002B36
:104800001BDB184A92F842616A46192EB8BF192676
:10481000002490460A20B3FBF0F100FB113342F86C
:10482000043B01340B460029F5D1DFF84490DFF852
:1048300044A023465D1E1BB93D600AB0BDE8F08769
:104840009C4204D049464FF4FA70FFF7ADFF58F888
:10485000253031465AF8230001F054F92B46E9E798
:1048600099060020000000206468000880010020F4
:1048700061410008C469000838B5114C23782BB198
:10488000104B1D7815B900F0BFFD25700E4B1B783D
:104890001A0713D1FCF776FF0C4B1B68DB0601D11E
:1048A00000F0EAFD0A4B93F845010A4B1A68824270
:1048B00004D01860BDE8384000F0ACBE38BD00BF81
:1048C0000507002004070020140700201807002017
:1048D000000000207C01002008B5012000F09AFEB5
:1048E0000D4B8022C3F8142CA3F5883342F6DF6207
:1048F0009A6242F20F72DA6201225A616FF001028B
:104900001A6109221A601A68D207FCD4034B80226C
:10491000C3F8002CFEE700BF00200140002000404B
:104920002DE9F04FAF48B04AB04CB149B14E95B007
:10493000121A01F05BFA00F0E9FEE37D0693AE4B3C
:1049400094F823201A7094F82730AC4A03EB8303C1
:104950009B001360AA4B94F836201A70FCF7B0FD48
:1049600000F024FE00F023FE00F0D0FCFFF7C4FBB3
:1049700048F64203C6F8443C41F28733C6F82C3C63
:104980008123C6F8003C3523C6F8043C4FF0804331
:104990003B22C3F8282400250422C3F82C54C3F872
:1049A00000240122C3F814248522C3F800248021A6
:1049B000FE2001F0D3FB4FF0E02341F64B525A6149
:1049C00007229D611A6194F83F308E4A079313784D
:1049D000002B00F0E580079B43B98B4B1B684FF41D
:1049E000DC7203F2B71393FBF2F30793874B5D6A14
:1049F0004FF0807215F0C04F5A621BD194F84230CC
:104A00007E2B40F0CF80824801F0C2F920EAE071AD
:104A100064298048A8BF642101F032F994F83E303F
:104A200043B17D4B079A7D491A60FA20FFF7BCFE1F
:104A3000FFF7D2FE237D0BB96C001ED5784C6F4D6D
:104A400042F6DF63A36240F6C313E36204232360EC
:104A500001270523676123606FF0010323612F6045
:104A60002369D80740F1A48000232B6023605F4BAB
:104A70006C4893F8421101F045F8FFF715FD142238
:104A8000002109A801F0C0F93223089314224FF441
:104A90007A7300210FA80A9301F0B6F94FF4C87396
:104AA0000E934FF416734FF0000A10934F4DCDF84C
:104AB00010A00223D34657460393D046D146049A0A
:104AC000E87E594BB3FBF0F3059340F6B8339A42B6
:104AD000697E18BF494B01EB810114BF1C6800249B
:104AE000890014BF4FF00A0C4FF0000CB8F1000F12
:104AF00008BF4FF00009002C40F0A080039B95F800
:104B00002320012B08BF022303933B4B19789142CA
:104B100008D0069931B91A70B8F1000F02D1FFF729
:104B2000C3FC354B1B78002B4BD0404B95F8220033
:104B30001C68C4F164048442A8BF04464FF0000816
:104B40002D4B1B78002B40F04082B8F1000F00F095
:104B50003E826B7D002B0CBF00234223069A002A65
:104B600000F03782059AB43A009200214FF4FA62BD
:104B7000204600F08BFD8323C6F8003C059BC6F859
:104B80002C3C8123C6F8340CC6F8380CC6F83C0C13
:104B9000C6F8003CB8F1000F00F04F82A14696E045
:104BA00030BF14E794F84211214800F0ABFF35E71D
:104BB00030BFFFF711FE2B68002B3FF451AF676148
:104BC0004EE71C4A1268052A05DD1B4A1268B2F539
:104BD000487F80F2EE8195F8224004EB8404A40023
:104BE000ACE700BF000000204801002000000020CA
:104BF0000010000800200140E006002010070020FF
:104C000004070020F40600202807002000100240BE
:104C100043000020006E0008800100206141000870
:104C200000100040EC670008C0D40100C00600205E
:104C30004200002000070020CC06002080F2D9802E
:104C400095F82430022B40F0BD80039B022B40F0EE
:104C5000BC80774BAA7D95F825001B780438002A84
:104C600008BF83F00103734A4443A4101370DFF8B4
:104C7000C881D8F80030002B40F0C480CCF100038C
:104C80000B44A34280F2C080A87F6B7F00EB8000C2
:104C9000800003EB830300909B0020464FF4FA62F0
:104CA000614400F0F3FC0446634B1B68002B00F0EA
:104CB0008281002C40F0D880604A116839B1B4215B
:104CC0004B4313605E4A92FBF3F35E4A13605E4A05
:104CD00013681BBB069B5949002B00F08781554880
:104CE0006C7D0378002B00F0768140F2144C40F28A
:104CF0005443002C08BF6346582446F6580CC6F8A7
:104D000018CCC6F81C4CC6F8203C2123C6F8143C2D
:104D10000378013313604FF416730B6001234FF0D7
:104D2000E0220221C2F8101D30BF484A127812F06A
:104D30000F0145D1049840F6B732904200F3A281AA
:104D4000079895F83E2042430A20424340480068B5
:104D5000824240F39B81049A013204926A8F002AB6
:104D600000F096813B49B1FBF2F23B49059309689B
:104D7000A2F5487208A800F0AFFC07EB204727EA2D
:104D8000E777A02F059BA8BFA027B5F84020002AF1
:104D900000F0808164214A433049059309680EA8D8
:104DA00000F09AFC0BEBA02B2BEAEB7BBBF5FA6F28
:104DB000059BA8BF4FF4FA6B0593FFF70DFD059B0C
:104DC00098467CE6032B7FF444AF95F8222095F8B3
:104DD0002630234902EB8202920003EB8303009208
:104DE0009B002046002200F051FC0123044603935F
:104DF000A4E60F4AAB7D127853400E4A137000238D
:104E0000039334E763463BE7A1EB0C02698F69B17A
:104E1000144BB3FBF1F3009320464FF47A73002157
:104E200000F034FC0024C8F800003DE79123F2E7CD
:104E3000D5060020F5060020F8060020D006002048
:104E400000879303CC060020FC06002014070020F6
:104E500028070020002D3101DC060020BC060020C0
:104E600030F8FFFF1516050072B68D490B7833B385
:104E70008C4FDFF834C23B689CF800C0581E3C23BE
:104E800090FBF3F2BCF1000F00F006810132062A1C
:104E900090FBF3FC03FB1C0308BF00220133D8F88E
:104EA000000043434FF08040C0F83C344FF6FF739E
:104EB000C0F82C3401231A44C0F814343A607B4BF8
:104EC00000271F607A4BC8F800701F70794B0F7075
:104ED00042F21078C3F80080FFF748F962B6414605
:104EE00008A800F0F5FB4FF00108B946069B43B156
:104EF0006D4B6C4A1B78116801338B421CBF002339
:104F000013606D4BA7EB0B000444186824EAE474AB
:104F100088B16A4B93FBF0F0694B2A7F186047F227
:104F20003051684BB3FBF2F34EF660220093059BC1
:104F300000F0ACFB0590EB7F95F8202060484FF423
:104F4000FA61009103EB83034FF47A714A439B00AB
:104F50000068002100F09AFB5B4B1B686FF01802A1
:104F6000534303F5FA639C42A8BF1C46504B1B7881
:104F70008442A8BF04460BBB95F82130DA1003F039
:104F8000070353450AF1010AC8BF0132BAF1080FFD
:104F900008BF4FF0000A4C4512DA444B1B68052B42
:104FA0007FF7CEADA9EB02094C453FF7C9AD4C46A2
:104FB000C6E51F469AE74FF0010897E70023DDE7B3
:104FC00091444C45FFF6BCADF1E74223C6E54346AC
:104FD000C4E5059AC8E540F2411C40F24553002C57
:104FE00008BF6346682445F6680C88E672B6374BFE
:104FF0001B6813602F4B42F210771F60344B0B601D
:10500000FFF7B4F82123C6F8143CD6F80C3C4FF057
:10501000804243F02003C6F80C3C01244FF6FF7396
:10502000C2F83C34C2F82C34C2F8144462B6394693
:1050300008A800F04DFB069F70E61A4B1B68FBB1F9
:1050400072B6D6F80C3C23F02003C6F80C3C4FF0A7
:1050500080430122C3F80C84C3F82C84C3F81424C1
:10506000FFF722FA114BC3F80080114B83F8008040
:10507000114BC3F80080124BC3F8008062B6434660
:10508000A1464CE6002B7FF469AED7E4049165E6B7
:1050900017467AE693468FE653431B1A3C33FEE6E7
:1050A000EC060020FC060020F5060020000700208A
:1050B000D4060020DC060020D006002000879303E1
:1050C000CC060020C0D40100C0060020E406002069
:1050D00000E1F505C0F57F43CAB2F93330B59B1A3C
:1050E000C1F307229B1A064A04460D1206201371CB
:1050F0001B12107054709170D570537130BD00BF89
:105100002C0700200368134403EB2323DBB210B504
:105110000360A2F17D03012B064806D80B685C1CD6
:105120000C607D24C45402F0DF020B685C1C0C6030
:10513000C25410BD2C07002037B500230C4605468D
:1051400001A968461022CDE90033FFF7DBFFEAB280
:105150006846FFF7D7FFC5F307226846FFF7D2FF7F
:10516000E2B26846FFF7CEFFC4F307226846FFF7B6
:10517000C9FFC4F307426846FFF7C4FF220E684622
:10518000FFF7C0FF009AD2436846D2B2FFF7BAFFDA
:10519000019803B030BD0000042830B402464CD161
:1051A000274B1978042948D158785B884FF6FB7152
:1051B00003448B4241D1234C94F837306FF00505FE
:1051C000591E00F00F0305FB0133013B052B34D8BA
:1051D0000109092907D00A290BD0082918BF002284
:1051E000104630BC7047184A32F8131030BCFFF735
:1051F00071BF013B042B04D8DFE803F0090B0E104C
:105200001200124B1B680A2128335943EEE7104B5A
:10521000F8E7104B1968E9E70F4BFBE70F4BF9E78D
:1052200094F838100E4B49081B6893FBF1F34FF6C6
:10523000FF719942A8BF1946D8E70022D0E700BF06
:105240002C07002000000020F0690008080700205B
:105250000C07002028070020BC060020B80600200C
:10526000CC060020022810B438D11E4B1A787E2AB2
:1052700034D11D495A7891F8373002F01F02013BB2
:105280009A422BD1194A1A481368062B04BF0023EF
:10529000136013685C1C30F813001460052B1DD8D4
:1052A000DFE803F003080A0C1214124B196810BC53
:1052B000FFF742BF104BF9E7104BF7E7104B1968A7
:1052C000CD235943C912F2E70E4BEFE791F838307E
:1052D0000D4A5B08116891FBF3F1E8E7002010BC70
:1052E000704700BF2C07002000000020440700206A
:1052F000FC690008080700200C0700202807002090
:10530000BC060020B8060020CC060020184A40F257
:105310001243C2F80838174B1978174B032917D0D6
:1053200004291CD0022901D1144A1A601A68104BB2
:10533000C2B1C822C3F8142842F21C02C3F80C28D8
:105340000F4B1049104A9963DA6359629A627047A9
:105350000E49196040F62301C2F80818E6E74FF439
:105360009071F9E78822C3F8142842F20802E5E7B1
:1053700000300140040700203C070020995100083C
:1053800000000240043801402C070020655200084C
:1053900070B5164CD4F80C6816F0400618D1144DB0
:1053A000D4F80038D4F80438686B124BC0F1100000
:1053B0001B68984760B16FF04003C4F8003842F2B0
:1053C0004803C4F80C389123EE612862EB6170BD8C
:1053D000064B42F21C02C3F80C2803F5504300228E
:1053E0001A6310225A6381221A63F0E700300140E9
:1053F000000002403C070020024B20225A6000229D
:10540000DA6170470000024038B5144DEB69DB07E4
:1054100023D4134B134C1B6829225343124A12689E
:105420002270124A1268A2701112114A6170126839
:10543000227111120F4AE1701268A271111261718A
:105440001A1509211B1320462372E27100F0FEF8A1
:105450000A2360722B629323EB6138BD0000024087
:10546000CC0600202C070020080700202807002079
:10547000BC060020B806002038B5354B1B78012B40
:105480000FD0042B10D0334B1B78002B43D0324A63
:105490001368591C1160032B57D8DFE803F0323D25
:1054A000424BFFF7B1FFEEE72C4DE86910F0010029
:1054B000E9D12B4B2B4C1A682B4BA0721B68CD21CA
:1054C0004A434B43C82121700A2161700821A17011
:1054D000D114D2122271DA14DB12A371234B627140
:1054E0001B68E1701A14E27109211A12A01C637280
:1054F000227200F0BBF80C23E0722B629323EB6165
:10550000C1E71B4B1B7843F4007372B6194A11684C
:1055100001B9136062B638BD174B1B7843F40063C2
:10552000F3E70F4B1B6829225343C3F3872343F44C
:105530008063EAE70C4B1B6829214B43C3F3073315
:10554000002143F4C0631160DFE70023DDE700BF03
:1055500004070020C406002040070020000002408D
:10556000280700202C070020BC060020B8060020D9
:1055700008070020C80600200C0700200A4B012263
:105580005A6103F58833D3F8102CD2070BD56FF08E
:105590000102C3F8102CD3F8342CD3F83C1CC3F808
:1055A000341CC3F83C2C70470010004070474FF08B
:1055B00090435A6942F400425A615A6842F40042E8
:1055C0005A601A6822F000421A60D3F8142442F09C
:1055D0002002C3F81424D3F8042442F02002C3F8B4
:1055E0000424D3F8002422F40062C3F80024D3F882
:1055F000142442F00802C3F81424D3F8042442F01F
:105600000802C3F80424D3F8002422F08002C3F86F
:105610000024704710F0010F4FF0904314BF4FF07B
:1056200000424FF4004210F0020F9A6114BF4FF491
:105630000012202210F0040FC3F8182414BF4FF4F6
:1056400000220822C3F818247047000010B5064A4B
:105650000346014400208B4200D110BD13F8014BDA
:105660006040105CF7E700BF226B000810B5064AE7
:105670000346014400208B4200D110BD13F8014BBA
:105680006040105CF7E700BF226A000810B50446CE
:105690008C421846029B0ADD9442BFBF641A1B1A53
:1056A0005C43521AAEBF184694FBF2F4001910BDC9
:1056B00000290BDB0368002BB8BF01FA02F3194481
:1056C0001341C91A016041FA02F070470020704787
:1056D0000023C0E90431704730B5D0E903548A1A79
:1056E00013196C42A342B8BF2346AB424469A8BF1A
:1056F0002B46C0E904310C1BD0E9001580686B43D0
:1057000001FB023300FB043030BD000070B5C34B19
:1057100093F83440012C00F062811D7D003D18BFDC
:1057200001255A7DD87D1D75111E18BF012159759F
:10573000997D003918BF01219975011E18BF0121FB
:10574000D975197E0129B8BF01211F29A8BF1F21C2
:105750001976597E59B1002A00F04381002840F0A3
:1057600040810529B8BF05211929A8BF19215976FB
:10577000997E1E7F0129B8BF01210F29A8BF0F21E3
:105780009976D97E1029B8BF10213029A8BF3021C1
:10579000B142D976B8BF31466029A8BF60211977D8
:1057A000597F9E7F0129B8BF01216429A8BF6421C8
:1057B000B1425977B8BF31466429A8BF64219977AF
:1057C000D97F93F823600129B8BF01216429A8BFBC
:1057D0006421D97793F820106429A8BF642183F845
:1057E000201093F821100129B8BF01216429A8BF16
:1057F000642183F8211093F822106429A8BF642142
:1058000083F82210002E00F0EE8012B1B0FA80F280
:105810005209012C93F8246083F8232000F0E580DE
:10582000002A08BF0322B242A8BF324683F82420D0
:1058300093F82520032AA8BF032283F8252093F894
:1058400026208A42B8BF0A46642AA8BF642283F889
:105850002620002D93F8272014BF002164218A42BE
:10586000A8BF0A4683F8272093F82820003A18BFDB
:10587000012283F828205A8DB2F5617FB8BF4FF41A
:10588000617240F26C718A42A8BF0A46D98D5A856E
:1058900002F1C805A942B8BF294640F63405A9421D
:1058A000A8BF29469D8DD9856432AA42A1F1640121
:1058B000B8BF2A469142A8BF11461A8E9985B2F503
:1058C000486F598EA8BF4FF448621A86C8328A4280
:1058D000B8BF0A4640F648518A42A8BF0A46052C7E
:1058E0005A862246A8BF0522022C83F834207ED98E
:1058F00093F83520032C14BF10210E21012AB8BFC4
:1059000001228A42A8BF0A4683F8352093F8362040
:10591000042A1146A8BF0421022A83F8361068D150
:1059200093F83720012AB8BF0122022AA8BF022219
:1059300083F8372093F8382022F00102022AB8BFFA
:105940000222642AA8BF642283F838205A8F5AB1F1
:10595000002865D140F2DC518A42B8BF0A4640F6C1
:10596000AC518A42A8BF0A465A8793F83C202AB114
:105970003C2AB8BF3C228C2AA8BF8C2283F83C204A
:10598000002283F83D2093F83E202AB11C2AB8BF9C
:105990001C22262AA8BF262283F83E2093F83F2007
:1059A000182AA8BF182283F83F2093F84221642ABE
:1059B000A8BF642283F8422193F84321642AA8BF38
:1059C000642283F8432193F84521002102F0070265
:1059D00083F8441183F84521A3F8401070BD254693
:1059E0009FE60021C3E6324613E700221BE70022B0
:1059F0008AE7032A08D193F83720012AB8BF012289
:105A00001C2AA8BF1C2293E7042C05D193F8372049
:105A1000042AA8BF04228BE7002289E700000020A7
:105A20000022A1E738B51E4B1B680BB1002038BD22
:105A30001C4B1B78002BF9D172B61B4B1B4A5A60CA
:105A400002F188325A604FF0FF32DA6002221A61A6
:105A5000174A5A6142221A61DA68D207FCD401223D
:105A60001A61144B1249144A0F481C4693420FD333
:105A70008023036162B6C36813F0140FD6D10D49B9
:105A80000B48121B00F0A2F9B0FA80F04009CEE7F3
:105A900033F8025B21F8025BC568ED07FCD4E5E74B
:105AA000D00600204807002000200240230167455F
:105AB00000100008000000204801002008B572B660
:105AC000054906484FF4A37200F090F962B6BDE8AC
:105AD0000840FFF7A7BF00BF78680008000000205B
:105AE000074B44F24002C3F8182C4022C3F81C2C88
:105AF00040F24442C3F8202C2122C3F8142C7047F2
:105B0000002001402DE9F74F0F460A2201A9064661
:105B100000F06CFA019BB34246D0A0F10A0140F2BA
:105B2000DD32914200F29F801E4643F6982898FB92
:105B3000F0F8002F00F097804C4B1868002840F0D8
:105B40009280DFF82C9199F8001051BB494CDFF896
:105B500028A1012389F80030FFF7C2FF45F268034E
:105B6000C4F8183C6823C4F81C3C40F24553C4F800
:105B7000203C0E23C4F8283C8B46354615F8012BF3
:105B8000AAB9002141F28733C4F8281CC4F82C3C80
:105B9000FFF7A6FF15F8010C89F80010B0FA80F0A5
:105BA000400903B0BDE8F08F4FF07D08C1E7A2F1D6
:105BB0006101062921D8633A00210732072092FBB0
:105BC000F0F0C0EBC000121A520070782B4B042A80
:105BD000C8BF02F1FF32232808BF0132594433F80D
:105BE000122042FA01F107F10502C4F82C1C08BF8B
:105BF000B51CC4F8342C00220BE0A2F141010629A7
:105C000002D8433A0121D8E75F2A1AD10022C4F80A
:105C1000342C2123C4F83C2C01A90A22C4F8143CDA
:105C2000284600F0E3F9019AAA421AD0411E6229DF
:105C3000A7D81546514600FB08F0FEF7B5FD2E46E5
:105C40009BE72B2A05D1BBF1000F9AD14FF0010B36
:105C5000F5E72D2A95D1BBF1000F92D04FF0000B44
:105C6000EDE70120E6E700209BE700BFD00600201B
:105C700048070020002001407D550008086A000800
:105C80002DE9F84302683A4B9A426ED1C368B3F1EA
:105C9000007F6AD14369B3F1807F66D1002964D067
:105CA000344B1B68002B60D1334E3578002D5CD10E
:105CB00001273770FFF714FF304A314C45F2680373
:105CC000C2F8183C6823C2F81C3C40F24553C2F8A5
:105CD000203C41F28733C2F8345CC2F83C5CC2F825
:105CE0002C3C2123C2F8143CA56203691DBA254B44
:105CF00003EB5503B3FBF5F3013BE36267612760F8
:105D0000436885681BBA2DBA18446FF00108054432
:105D10004FF0830E78274FF0810C2369DB07FCD509
:105D20002B1A002BC4F810801ADD10F9013BC2F8C1
:105D300000EC03F18009C3F17F0301FB09F94B4338
:105D400007FB09F97B434FEA69395B1309F1420903
:105D50004233C2F8349CC2F83C3CC2F800CCDCE7C9
:105D600000212160FFF7BCFE3170BDE8F88300BF61
:105D70002E736E64D00600204807002000200140EA
:105D800000100040000E27070028B8BF40427047AF
:105D90000A22002100F02AB9931E222B10B50C46CE
:105DA00004D900230B701C46204610BD0A2A09D1D5
:105DB000002807DA2D230B7040420121214400F016
:105DC0001FF9F1E70021F9E7FFF7E6BF10B5013948
:105DD0000244904201D1002005E0037811F8014F00
:105DE000A34201D0181B10BD0130F2E70A449142D2
:105DF00000F1FF3300D1704710B511F8014B03F8E3
:105E0000014F9142F9D110BD02440346934200D1A3
:105E1000704703F8011BF9E7034611F8012B1846F8
:105E200003F8012B002AF8D17047000030B50B4D64
:105E3000044614F8013B5A5D02F00302012A11F8EE
:105E4000012BA85C00F0030008BF2033012808BF25
:105E50002032981A01D1002AEBD130BD486C0008DD
:105E600010B50B4662B1013A08D013F8014B00F8A7
:105E7000014B002CF7D1581A013810BD00220270D6
:105E800013F8012B002AFBD1F5E7034613F8012B89
:105E9000002AFBD1181A0138704702460023006817
:105EA00000F000B8F0B508B9106888B10446204683
:105EB00014F8015B0F4617F8016B1EB965B9156040
:105EC000284605E0B542F6D1002BF0D114600370EE
:105ED000F0BD1C460CE015B914F8013B0E4616F84F
:105EE000015BAB42F7D1002BF3D0002304F8013C57
:105EF0001460EDE7012B2DE9F047804601D0242BFB
:105F000006D900F0BFF8162303600020BDE8F08733
:105F1000354F0D46284615F8014BE65D16F008068C
:105F2000F8D12D2C2FD12C780126851C002B57D091
:105F3000102B09D1302C07D1287800F0DF00582829
:105F400049D16C781023023506F1004E0EF1FF3E68
:105F50000027BEFBF3F9384603FB19EAA4F1300C25
:105F6000BCF1090F14D86446A34222DD002F1DDBCB
:105F700081451BD301D1A24518DB00FB034001275B
:105F800015F8014BEAE72B2C04BF2C78851CCDE7D4
:105F9000A4F1410CBCF1190F01D8373CE4E7A4F19E
:105FA000610CBCF1190F04D8573CDDE74FF0FF3707
:105FB000E6E7002F07DA2223C8F800307046002AEF
:105FC000A4D0691E05E006B14042002A9ED0002FF1
:105FD000F7D111609AE73024002BB5D10823B3E73D
:105FE000302CA9D00A23AFE7486C000813460A46B4
:105FF000014602480068FFF77DBF00BF9C010020FA
:10600000F0B51F4C8BB005460B466E4604F1200CD4
:1060100020686168374603C7083464453E46F7D1B7
:1060200021793971911E2068386022294FF00001D2
:1060300004D919700B4618460BB0F0BD581E8446A3
:10604000B5FBF2F70DF1280E02FB175676440C460D
:1060500016F8286C0CF8016F2E46B24201F10101CE
:106060003D46EDD900225A541919A51AAA42E2DA7E
:1060700010F8015F0E780670013201F80159F4E75B
:10608000226C0008014B1868704700BF9C0100207B
:10609000FEE7704710B5164B164A17498B4218D3C6
:1060A0000021164A934217D38023154A9B0011689A
:1060B000144C0B431360144B9C420FD3134C144BE2
:1060C0009C420ED3FEF72CFC124C134B9C420BD37C
:1060D00010BD01CA01C3E1E702C3E3E708CC98475A
:1060E000E9E708CC9847EAE708CC9847EDE7C046CF
:1060F00048010020486D0008000200204C070020E5
:1061000014ED00E0486D0008486D0008486D000877
:10611000486D0008486D0008486D0008014B024AB0
:106120001A60FEE70CED00E00400FA05044A43099A
:106130009B009B181F2210401E3A82401A60704735
:1061400000E100E0044A43099B009B181F22104015
:106150001E3A82401A60704780E200E010B51F28A6
:1061600012D90F2318400438C0B28308084A9B0094
:106170001824C0002040E734844081409B181A68EE
:10618000A2431143196010BD8308024A9B00EFE748
:1061900018ED00E000E400E0C1180400E11804007C
:1061A000D1180400900197019E01A501AC01B30133
:1061B000BA01C101C801CF01D501DC01E301EA0147
:1061C000F101F801FE0105020C02120219021F0280
:1061D00026022C02330239023F0246024C025202CE
:1061E00058025E0264026A02700275027B0281023A
:1061F00086028C02910296029C02A102A602AB02C8
:10620000B002B502B902BE02C202C702CB02CF027F
:10621000D402D802DC02DF02E302E702EA02EE0265
:10622000F102F402F802FB02FD020003030305037E
:1062300008030A030C030F031103120314031603CC
:10624000170319031A031B031C031D031E031E035C
:106250001F031F03200320032003200320031F0329
:106260001F031E031E031D031C031B031A03190334
:10627000170316031403120311030F030C030A037D
:106280000803050303030003FD02FB02F802F40206
:10629000F102EE02EA02E702E302DF02DC02D802C8
:1062A000D402CF02CB02C702C202BE02B902B502BB
:1062B000B002AB02A602A1029C02960291028C02DD
:1062C000860281027B02750270026A0264025E022B
:1062D000580252024C0246023F02390233022C029B
:1062E00026021F02190212020C020502FE01F80129
:1062F000F101EA01E301DC01D501CF01C801C101CF
:10630000BA01B301AC01A5019E0197019001890179
:1063100082017B0174016D0166015F015801510129
:106320004B0144013D0136012F01280122011B01CF
:1063300014010E0107010101FA00F400ED00E7006D
:10634000E100DA00D400CE00C800C200BC00B600F4
:10635000B000AB00A5009F009A0094008F008A0057
:1063600084007F007A00750070006B006700620097
:106370005E005900550051004C00480044004100A7
:106380003D003900360032002F002C002800250087
:10639000230020001D001B0018001600140011002F
:1063A0000F000E000C000A0009000700060005009F
:1063B00004000300020002000100010000000000D0
:1063C00000000000000001000100020002000300C4
:1063D000040005000600070009000A000C000E007A
:1063E0000F0011001400160018001B001D002000F3
:1063F0002300250028002C002F0032003600390031
:106400003D004100440048004C0051005500590037
:106410005E00620067006B00700075007A007F000C
:1064200084008A008F0094009A009F00A500AB00B2
:10643000B000B600BC00C200C800CE00D400DA0034
:10644000E100E700ED00F400FA00010107010E0190
:1064500014011B01220128012F0136013D014401D5
:106460004B01510158015F0166016D0174017B010F
:10647000820189012E00300020090D0A0055736148
:1064800067653A0A696E666F0A73686F770A6765AF
:1064900074203C706172616D3E0A736574203C70BB
:1064A0006172616D3E203C76616C75653E0A736178
:1064B00076650A72657365740A706C6179203C6D4B
:1064C000757369633E205B3C766F6C756D653E5DF0
:1064D0000A7468726F74203C76616C75653E0A625E
:1064E0006565700A004553436170653332207265FB
:1064F0007600205B005D0A54656D703A2000432CE5
:10650000206578742000430A566F6C743A20005658
:106510000A437572723A2000410A4373756D3A203E
:10652000006D41680A4552504D3A200061726D007D
:1065300064616D7000726576646972006272757371
:106540006865640074696D696E670073696E655F84
:1065500072616E67650073696E655F706F776572F3
:1065600000667265715F6D696E00667265715F6D60
:10657000617800647574795F6D696E006475747913
:106580005F6D617800647574795F73707570006415
:106590007574795F72616D7000647574795F726192
:1065A000746500647574795F647261670064757402
:1065B000795F6C6F636B007468726F745F6D6F648A
:1065C00065007468726F745F726576007468726FCC
:1065D000745F62726B007468726F745F73657400CD
:1065E0007468726F745F63616C007468726F745F5B
:1065F0006D696E007468726F745F6D6964007468B1
:10660000726F745F6D617800616E616C6F675F6D52
:10661000696E00616E616C6F675F6D617800696EB5
:106620007075745F6D6F646500696E7075745F631B
:106630006869640074656C656D5F6D6F6465007496
:10664000656C656D5F706869640074656C656D5F2D
:10665000706F6C65730070726F745F7374616C6CD3
:106660000070726F745F74656D700070726F745F2C
:1066700073656E730070726F745F766F6C74007008
:10668000726F745F63656C6C730070726F745F63BC
:10669000757272006D7573696300766F6C756D65E8
:1066A00000626561636F6E00626563006C65640023
:1066B0004F4B0A004552524F520A0068656C7000F9
:1066C000696E666F0073686F770067657400736149
:1066D000766500726573657400706C61790074682A
:1066E000726F74006265657000000000BB66000890
:1066F000C0660008C5660008CA660008DC650008B8
:10670000CE660008D3660008D9660008DE66000879
:10671000E4660008000000002C65000830650008F1
:10672000356500083C650008446500084B650008B5
:1067300056650008616500086A6500087365000811
:106740007C650008856500088F650008996500086C
:10675000A3650008AD650008B7650008C2650008BC
:10676000CC650008D6650008E0650008EA65000809
:10677000F4650008FE650008086600081366000856
:106780001E66000829660008346600083F66000897
:106790004A66000856660008616600086B660008D5
:1067A000756600087F6600088A660008946600081F
:1067B0009A660008A1660008A8660008AC66000892
:1067C00000000000191B12131D1516171A090A0BD9
:1067D0001E0D0E0F43C323A363E353D333B373F3ED
:1067E0004BCB2BAB6BEB5BDB3BBB7BFB47430063D8
:1067F0003600462332453244324332004723412398
:106800004723412347233200472341234723412382
:106810004623324723320047234123472341234560
:106820003246233247233200472341234723412363
:10683000443245324623324723320047234123471F
:106840002341234332443245324623324723320028
:10685000454700464100474200414223006144470A
:10686000450000005068000853680008566800089A
:10687000596800085D680008EA320E0248414B5230
:106880004332000000000000000000000101000091
:10689000100008183001640F001E000000006400A2
:1068A0000100E803DC05D0076400800C0000000054
:1068B0000E0000000000000000006466612300007C
:1068C00000000000000000000000000000000000C8
:1068D00000000000000000000000000000000000B8
:1068E00000000000000000000000000000000000A8
:1068F0000000000000000000000000000000000098
:106900000000000000000000000000000000000087
:106910000000000000000000000000000000000077
:106920000000000000000000000000000000000067
:106930000000000000000000000000000000000057
:106940000000000000000000000000000000000047
:106950000000000000000000000000000000000037
:106960000000000000000000000000000000000027
:106970000000000000000000000000000000000017
:106980000000000000000000000000000000000007
:1069900000000000000000000000000000000000F7
:1069A00000000000000000000000000000000000E7
:1069B000000000000000000000001932000035193E
:1069C0002B321E2CEF670008F9670008F7670008F4
:1069D000F5670008F2670008FC670008086800080F
:1069E00017680008286800083B68000800000000DD
:1069F000010201020302050206020202700B0004FA
:106A000010020002300B0005B73B5D3833353832D9
:106A1000652FBC2C3A2ADB279E2582238321A11FC8
:106A2000DB1D00D57FAAFE2B815429FC5683D7029B
:106A3000A87D52872DF8AC79D3067BAE04D1855062
:106A4000FA2FA471DB0E5A8F25F08D58F22773A60A
:106A50000CD9F623895C08DD77A2DF0AA07521F442
:106A60005E8B9D48E23763B61CC9B461CB1E4A9F5A
:106A700035E0CF1AB06531E44E9BE633994C18CD22
:106A800067B239EC4693C712B86D10C56FBAEE3BCA
:106A900091446BBE14C19540EA3F42973DE8BC6902
:106AA000C316EF3A904511C46EBBC613B96C38EDEE
:106AB0004792BD68C21743963CE99441EB3E6ABFDA
:106AC00015C04B9E34E1B560CA1F62B71DC89C4912
:106AD000E33619CC66B3E732984D30E54F9ACE1BBA
:106AE000B16472A70DD88C59F3265B8E24F1A57082
:106AF000DA0F20F55F8ADE0BA17409DC76A3F7229A
:106B0000885DD603A97C28FD5782FF2A805501D4D1
:106B10007EAB8451FB2E7AAF05D0AD78D207538679
:106B20002CF900070E091C1B1215383F363124239F
:106B30002A2D70777E796C6B6265484F46415453BD
:106B40005A5DE0E7EEE9FCFBF2F5D8DFD6D1C4C32D
:106B5000CACD90979E998C8B8285A8AFA6A1B4B31D
:106B6000BABDC7C0C9CEDBDCD5D2FFF8F1F6E3E48D
:106B7000EDEAB7B0B9BEABACA5A28F88818693947D
:106B80009D9A2720292E3B3C35321F1811160304ED
:106B90000D0A5750595E4B4C45426F6861667374DD
:106BA0007D7A898E878095929B9CB1B6BFB8ADAA3D
:106BB000A3A4F9FEF7F0E5E2EBECC1C6CFC8DDDA3D
:106BC000D3D4696E676075727B7C51565F584D4AAD
:106BD0004344191E171005020B0C21262F283D3A9D
:106BE00033344E49404752555C5B7671787F6A6D0D
:106BF00064633E39303722252C2B0601080F1A1DFD
:106C00001413AEA9A0A7B2B5BCBB9691989F8A8D6C
:106C10008483DED9D0D7C2C5CCCBE6E1E8EFFAFD5C
:106C2000F4F33031323334353637383961626364E6
:106C300065666768696A6B6C6D6E6F70717273748C
:106C400075767778797A0000202020202020202077
:106C5000202828282828202020202020202020200C
:106C6000202020202020202088101010101010102C
:106C70001010101010101010040404040404040474
:106C80000404101010101010104141414141410105
:106C900001010101010101010101010101010101E4
:106CA00001010110101010101042424242424202F3
:106CB00002020202020202020202020202020202B4
:106CC000020202101010102000000000000000005E
:106CD00000000000000000000000000000000000B4
:106CE00000000000000000000000000000000000A4
:106CF0000000000000000000000000000000000094
:106D00000000000000000000000000000000000083
:106D10000000000000000000000000000000000073
:106D20000000000000000000000000000000000063
:106D30000000000000000000000000000000000053
:086D400000000000000000004B
:106D4800FFFFFFFFFFFFFFFF0000FFFF0000FFFF47
:106D5800FFFF0000FFFF0000FFFFFFFF0000FFFF35
:106D68000000FFFF0000FFFFFFFFFFFF0000000023
:106D780000000000FFFFFFFFFFFFFFFFFFFFFFFF17
:106D8800FFFFFFFFFFFFFFFFFFFFFFFFFFFFFFFF0B
:106D9800E40C0000A001002000000000000000003A
:106DA80000000000000000000000000000000000DB
:106DB80000000000000000000000000000000000CB
:106DC80000000000000000000000000000000000BB
:106DD80000000000000000000000000000000000AB
:106DE800000000000000000000000000000000009B
:086DF800000000000000000093
:0400000508006095FA
:00000001FF
